******************************************************************************
             TMS320C2000 Linker PC v18.12.5                    
******************************************************************************
>> Linked Thu Oct 22 14:14:36 2020

OUTPUT FILE NAME:   <empty_driverlib_project.out>
ENTRY POINT SYMBOL: "code_start"  address: 00080000


MEMORY CONFIGURATION

         name            origin    length      used     unused   attr    fill
----------------------  --------  ---------  --------  --------  ----  --------
PAGE 0:
  RAMM0                 000000f3   0000030d  00000000  0000030d  RWIX
  RAMLS0                00008000   00000800  00000130  000006d0  RWIX
  RAMLS1                00008800   00000800  00000000  00000800  RWIX
  RAMLS2                00009000   00000800  00000000  00000800  RWIX
  RAMLS3                00009800   00000800  00000000  00000800  RWIX
  RAMLS4                0000a000   00000800  00000000  00000800  RWIX
  BEGIN                 00080000   00000002  00000002  00000000  RWIX
  FLASH_BANK0_SEC0      00080002   00000ffe  00000000  00000ffe  RWIX
  FLASH_BANK0_SEC1      00081000   00001000  00000144  00000ebc  RWIX
  FLASH_BANK0_SEC2      00082000   00001000  0000087f  00000781  RWIX
  FLASH_BANK0_SEC3      00083000   00001000  00000000  00001000  RWIX
  FLASH_BANK0_SEC4      00084000   00001000  00000291  00000d6f  RWIX
  FLASH_BANK0_SEC5      00085000   00001000  00000000  00001000  RWIX
  FLASH_BANK0_SEC6      00086000   00001000  00000000  00001000  RWIX
  FLASH_BANK0_SEC7      00087000   00001000  00000000  00001000  RWIX
  FLASH_BANK0_SEC8      00088000   00001000  00000000  00001000  RWIX
  FLASH_BANK0_SEC9      00089000   00001000  00000000  00001000  RWIX
  FLASH_BANK0_SEC10     0008a000   00001000  00000000  00001000  RWIX
  FLASH_BANK0_SEC11     0008b000   00001000  00000000  00001000  RWIX
  FLASH_BANK0_SEC12     0008c000   00001000  00000000  00001000  RWIX
  FLASH_BANK0_SEC13     0008d000   00001000  00000000  00001000  RWIX
  FLASH_BANK0_SEC14     0008e000   00001000  00000000  00001000  RWIX
  FLASH_BANK0_SEC15     0008f000   00001000  00000000  00001000  RWIX
  FLASH_BANK1_SEC0      00090000   00001000  00000000  00001000  RWIX
  FLASH_BANK1_SEC1      00091000   00001000  00000000  00001000  RWIX
  FLASH_BANK1_SEC2      00092000   00001000  00000000  00001000  RWIX
  FLASH_BANK1_SEC3      00093000   00001000  00000000  00001000  RWIX
  FLASH_BANK1_SEC4      00094000   00001000  00000000  00001000  RWIX
  FLASH_BANK1_SEC5      00095000   00001000  00000000  00001000  RWIX
  FLASH_BANK1_SEC6      00096000   00001000  00000000  00001000  RWIX
  FLASH_BANK1_SEC7      00097000   00001000  00000000  00001000  RWIX
  FLASH_BANK1_SEC8      00098000   00001000  00000000  00001000  RWIX
  FLASH_BANK1_SEC9      00099000   00001000  00000000  00001000  RWIX
  FLASH_BANK1_SEC10     0009a000   00001000  00000000  00001000  RWIX
  FLASH_BANK1_SEC11     0009b000   00001000  00000000  00001000  RWIX
  FLASH_BANK1_SEC12     0009c000   00001000  00000000  00001000  RWIX
  FLASH_BANK1_SEC13     0009d000   00001000  00000000  00001000  RWIX
  FLASH_BANK1_SEC14     0009e000   00001000  00000000  00001000  RWIX
  FLASH_BANK1_SEC15     0009f000   00000ff0  00000000  00000ff0  RWIX
  RESET                 003fffc0   00000002  00000000  00000002  RWIX

PAGE 1:
  BOOT_RSVD             00000002   000000f1  00000000  000000f1  RWIX
  RAMM1                 00000400   000003f8  00000100  000002f8  RWIX
  RAMLS5                0000a800   00000800  0000000a  000007f6  RWIX
  RAMLS6                0000b000   00000800  00000000  00000800  RWIX
  RAMLS7                0000b800   00000800  00000000  00000800  RWIX
  RAMGS0                0000c000   00002000  00000000  00002000  RWIX
  RAMGS1                0000e000   00002000  00000000  00002000  RWIX
  RAMGS2                00010000   00002000  00000000  00002000  RWIX
  RAMGS3                00012000   00001ff8  00000000  00001ff8  RWIX


SECTION ALLOCATION MAP

 output                                  attributes/
section   page    origin      length       input sections
--------  ----  ----------  ----------   ----------------
codestart 
*          0    00080000    00000002     
                  00080000    00000002     f28004x_codestartbranch.obj (codestart)

.cinit     0    00081130    00000014     
                  00081130    00000009     (.cinit..data.load) [load image, compression = lzss]
                  00081139    00000001     --HOLE-- [fill = 0]
                  0008113a    00000004     (__TI_handler_table)
                  0008113e    00000002     --HOLE-- [fill = 0]
                  00081140    00000004     (__TI_cinit_table)

.reset     0    003fffc0    00000000     DSECT

.stack     1    00000400    00000100     UNINITIALIZED
                  00000400    00000100     --HOLE--

.init_array 
*          0    00081000    00000000     UNINITIALIZED

.data      1    0000a800    0000000a     UNINITIALIZED
                  0000a800    00000006     rts2800_fpu32_eabi.lib : exit.c.obj (.data)
                  0000a806    00000002                            : _lock.c.obj (.data:_lock)
                  0000a808    00000002                            : _lock.c.obj (.data:_unlock)

.const     0    00084000    00000291     
                  00084000    000000bf     driverlib_eabi.lib : flash.obj (.const:.string)
                  000840bf    00000001     --HOLE-- [fill = 0]
                  000840c0    000000be                        : sysctl.obj (.const:.string)
                  0008417e    000000bc                        : gpio.obj (.const:.string)
                  0008423a    00000044     empty_driverlib_main.obj (.const:.string)
                  0008427e    00000013     device.obj (.const:.string)

.TI.ramfunc 
*          0    00081000    00000130     RUN ADDR = 00008000
                  00081000    00000044     driverlib_eabi.lib : flash.obj (.TI.ramfunc:Flash_initModule)
                  00081044    0000002d                        : flash.obj (.TI.ramfunc:Flash_setBankPowerMode)
                  00081071    00000026                        : flash.obj (.TI.ramfunc:Flash_setWaitstates)
                  00081097    0000001e                        : flash.obj (.TI.ramfunc:Flash_setPumpPowerMode)
                  000810b5    00000018                        : flash.obj (.TI.ramfunc:Flash_disableCache)
                  000810cd    00000018                        : flash.obj (.TI.ramfunc:Flash_disablePrefetch)
                  000810e5    00000018                        : flash.obj (.TI.ramfunc:Flash_enableCache)
                  000810fd    00000018                        : flash.obj (.TI.ramfunc:Flash_enablePrefetch)
                  00081115    00000017                        : flash.obj (.TI.ramfunc:Flash_enableECC)
                  0008112c    00000004                        : sysctl.obj (.TI.ramfunc)

.text      0    00082000    0000087f     
                  00082000    000001a8     device.obj (.text)
                  000821a8    000000b6     driverlib_eabi.lib : sysctl.obj (.text:SysCtl_setClock)
                  0008225e    0000009b                        : sysctl.obj (.text:SysCtl_isPLLValid)
                  000822f9    0000007b     empty_driverlib_main.obj (.text)
                  00082374    0000005b     driverlib_eabi.lib : sysctl.obj (.text:SysCtl_selectOscSource)
                  000823cf    00000056                        : sysctl.obj (.text:DCC_setCounterSeeds)
                  00082425    00000052                        : gpio.obj (.text:GPIO_setPadConfig)
                  00082477    00000051                        : sysctl.obj (.text:SysCtl_getClock)
                  000824c8    0000003d                        : interrupt.obj (.text:Interrupt_initModule)
                  00082505    0000003b                        : gpio.obj (.text:GPIO_setAnalogMode)
                  00082540    00000031                        : gpio.obj (.text:GPIO_setDirectionMode)
                  00082571    00000031     rts2800_fpu32_eabi.lib : copy_decompress_lzss.c.obj (.text:decompress:lzss)
                  000825a2    0000002b                            : autoinit.c.obj (.text:__TI_auto_init_nobinit_nopinit)
                  000825cd    00000029                            : exit.c.obj (.text)
                  000825f6    00000025     driverlib_eabi.lib : sysctl.obj (.text:DCC_enableSingleShotMode)
                  0008261b    00000024                        : sysctl.obj (.text:SysCtl_selectXTAL)
                  0008263f    00000022                        : sysctl.obj (.text:SysCtl_pollX1Counter)
                  00082661    00000020                        : interrupt.obj (.text:Interrupt_initVectorTable)
                  00082681    0000001f                        : sysctl.obj (.text:DCC_setCounter1ClkSource)
                  000826a0    0000001d                        : sysctl.obj (.text:DCC_setCounter0ClkSource)
                  000826bd    0000001d     rts2800_fpu32_eabi.lib : memcpy.c.obj (.text)
                  000826da    0000001a     driverlib_eabi.lib : sysctl.obj (.text:SysCtl_getLowSpeedClock)
                  000826f4    0000001a                        : sysctl.obj (.text:SysCtl_selectXTALSingleEnded)
                  0008270e    00000017                        : sysctl.obj (.text:DCC_disableDoneSignal)
                  00082725    00000017                        : sysctl.obj (.text:DCC_enableDoneSignal)
                  0008273c    00000017                        : sysctl.obj (.text:SysCtl_enablePeripheral)
                  00082753    00000017     rts2800_fpu32_eabi.lib : boot28.asm.obj (.text)
                  0008276a    00000016     driverlib_eabi.lib : sysctl.obj (.text:DCC_clearDoneFlag)
                  00082780    00000016                        : sysctl.obj (.text:DCC_clearErrorFlag)
                  00082796    00000016                        : sysctl.obj (.text:DCC_disableErrorSignal)
                  000827ac    00000016                        : sysctl.obj (.text:DCC_enableErrorSignal)
                  000827c2    00000014                        : sysctl.obj (.text:DCC_disableModule)
                  000827d6    00000014                        : sysctl.obj (.text:DCC_enableModule)
                  000827ea    00000014                        : gpio.obj (.text:GPIO_isPinValid)
                  000827fe    00000010                        : sysctl.obj (.text:DCC_isBaseValid)
                  0008280e    00000010                        : flash.obj (.text:Flash_isCtrlBaseValid)
                  0008281e    00000010                        : flash.obj (.text:Flash_isECCBaseValid)
                  0008282e    0000000e                        : interrupt.obj (.text:Interrupt_defaultHandler)
                  0008283c    0000000d                        : interrupt.obj (.text:Interrupt_disableMaster)
                  00082849    0000000c     rts2800_fpu32_eabi.lib : args_main.c.obj (.text)
                  00082855    0000000b     driverlib_eabi.lib : sysctl.obj (.text:SysCtl_isMCDClockFailureDetected)
                  00082860    00000009     rts2800_fpu32_eabi.lib : _lock.c.obj (.text)
                  00082869    00000008                            : copy_decompress_none.c.obj (.text:decompress:none)
                  00082871    00000007     driverlib_eabi.lib : sysctl.obj (.text:SysCtl_resetMCD)
                  00082878    00000002                        : interrupt.obj (.text:Interrupt_illegalOperationHandler)
                  0008287a    00000002                        : interrupt.obj (.text:Interrupt_nmiHandler)
                  0008287c    00000002     rts2800_fpu32_eabi.lib : pre_init.c.obj (.text)
                  0008287e    00000001                            : startup.c.obj (.text)

MODULE SUMMARY

       Module                        code   ro data   rw data
       ------                        ----   -------   -------
    .\
       empty_driverlib_main.obj      123    68        0      
    +--+-----------------------------+------+---------+---------+
       Total:                        123    68        0      
                                                             
    .\device\
       device.obj                    424    19        0      
       f28004x_codestartbranch.obj   2      0         0      
    +--+-----------------------------+------+---------+---------+
       Total:                        426    19        0      
                                                             
    C:\ti\c2000\C2000Ware_3_02_00_00\driverlib\f28004x\driverlib\ccs\Debug\driverlib_eabi.lib
       sysctl.obj                    1053   190       0      
       flash.obj                     632    191       0      
       gpio.obj                      210    188       0      
       interrupt.obj                 124    0         0      
    +--+-----------------------------+------+---------+---------+
       Total:                        2019   569       0      
                                                             
    C:\ti\ccs1000\ccs\tools\compiler\ti-cgt-c2000_18.12.5.LTS\lib\rts2800_fpu32_eabi.lib
       copy_decompress_lzss.c.obj    49     0         0      
       exit.c.obj                    41     0         6      
       autoinit.c.obj                43     0         0      
       memcpy.c.obj                  29     0         0      
       boot28.asm.obj                23     0         0      
       _lock.c.obj                   9      0         4      
       args_main.c.obj               12     0         0      
       copy_decompress_none.c.obj    8      0         0      
       pre_init.c.obj                2      0         0      
       startup.c.obj                 1      0         0      
    +--+-----------------------------+------+---------+---------+
       Total:                        217    0         10     
                                                             
       Stack:                        0      0         256    
       Linker Generated:             0      17        0      
    +--+-----------------------------+------+---------+---------+
       Grand Total:                  2785   673       266    


LINKER GENERATED COPY TABLES

__TI_cinit_table @ 00081140 records: 1, size/record: 4, table size: 4
	.data: load addr=00081130, load size=00000009 bytes, run addr=0000a800, run size=0000000a bytes, compression=lzss


LINKER GENERATED HANDLER TABLE

__TI_handler_table @ 0008113a records: 2, size/record: 2, table size: 4
	index: 0, handler: __TI_decompress_lzss
	index: 1, handler: __TI_decompress_none


GLOBAL DATA SYMBOLS: SORTED BY DATA PAGE

address     data page           name
--------    ----------------    ----
00000400      10 (00000400)     __stack

0000a800     2a0 (0000a800)     __TI_enable_exit_profile_output
0000a802     2a0 (0000a800)     __TI_cleanup_ptr
0000a804     2a0 (0000a800)     __TI_dtors_ptr
0000a806     2a0 (0000a800)     _lock
0000a808     2a0 (0000a800)     _unlock


GLOBAL SYMBOLS: SORTED ALPHABETICALLY BY Name 

page  address   name                           
----  -------   ----                           
0     000825cd  C$$EXIT                        
0     000820b4  Device_enableAllPeripherals    
0     00082052  Device_init                    
0     00082191  Device_initGPIO                
0     00008000  Flash_initModule               
0     00082505  GPIO_setAnalogMode             
0     00082540  GPIO_setDirectionMode          
0     00082425  GPIO_setPadConfig              
0     000824c8  Interrupt_initModule           
0     00082661  Interrupt_initVectorTable      
0     00081130  RamfuncsLoadEnd                
abs   00000130  RamfuncsLoadSize               
0     00081000  RamfuncsLoadStart              
0     00008130  RamfuncsRunEnd                 
abs   00000130  RamfuncsRunSize                
0     00008000  RamfuncsRunStart               
0     0000812c  SysCtl_delay                   
0     00082477  SysCtl_getClock                
0     000826da  SysCtl_getLowSpeedClock        
0     0008225e  SysCtl_isPLLValid              
0     00082374  SysCtl_selectOscSource         
0     0008261b  SysCtl_selectXTAL              
0     000826f4  SysCtl_selectXTALSingleEnded   
0     000821a8  SysCtl_setClock                
0     00081140  __TI_CINIT_Base                
0     00081144  __TI_CINIT_Limit               
0     0008113a  __TI_Handler_Table_Base        
0     0008113e  __TI_Handler_Table_Limit       
1     00000500  __TI_STACK_END                 
abs   00000100  __TI_STACK_SIZE                
0     000825a2  __TI_auto_init_nobinit_nopinit 
1     0000a802  __TI_cleanup_ptr               
0     00082571  __TI_decompress_lzss           
0     00082869  __TI_decompress_none           
1     0000a804  __TI_dtors_ptr                 
1     0000a800  __TI_enable_exit_profile_output
abs   ffffffff  __TI_pprof_out_hndl            
abs   ffffffff  __TI_prof_data_size            
abs   ffffffff  __TI_prof_data_start           
n/a   UNDEFED   __c_args__                     
0     000821a1  __error__                      
1     00000400  __stack                        
0     00082849  _args_main                     
0     00082753  _c_int00                       
1     0000a806  _lock                          
0     00082868  _nop                           
0     00082864  _register_lock                 
0     00082860  _register_unlock               
0     0008287e  _system_post_cinit             
0     0008287c  _system_pre_init               
1     0000a808  _unlock                        
0     000825cd  abort                          
0     00080000  code_start                     
0     000825cf  exit                           
0     00082335  main                           
0     000826bd  memcpy                         


GLOBAL SYMBOLS: SORTED BY Symbol Address 

page  address   name                           
----  -------   ----                           
0     00008000  Flash_initModule               
0     00008000  RamfuncsRunStart               
0     0000812c  SysCtl_delay                   
0     00008130  RamfuncsRunEnd                 
0     00080000  code_start                     
0     00081000  RamfuncsLoadStart              
0     00081130  RamfuncsLoadEnd                
0     0008113a  __TI_Handler_Table_Base        
0     0008113e  __TI_Handler_Table_Limit       
0     00081140  __TI_CINIT_Base                
0     00081144  __TI_CINIT_Limit               
0     00082052  Device_init                    
0     000820b4  Device_enableAllPeripherals    
0     00082191  Device_initGPIO                
0     000821a1  __error__                      
0     000821a8  SysCtl_setClock                
0     0008225e  SysCtl_isPLLValid              
0     00082335  main                           
0     00082374  SysCtl_selectOscSource         
0     00082425  GPIO_setPadConfig              
0     00082477  SysCtl_getClock                
0     000824c8  Interrupt_initModule           
0     00082505  GPIO_setAnalogMode             
0     00082540  GPIO_setDirectionMode          
0     00082571  __TI_decompress_lzss           
0     000825a2  __TI_auto_init_nobinit_nopinit 
0     000825cd  C$$EXIT                        
0     000825cd  abort                          
0     000825cf  exit                           
0     0008261b  SysCtl_selectXTAL              
0     00082661  Interrupt_initVectorTable      
0     000826bd  memcpy                         
0     000826da  SysCtl_getLowSpeedClock        
0     000826f4  SysCtl_selectXTALSingleEnded   
0     00082753  _c_int00                       
0     00082849  _args_main                     
0     00082860  _register_unlock               
0     00082864  _register_lock                 
0     00082868  _nop                           
0     00082869  __TI_decompress_none           
0     0008287c  _system_pre_init               
0     0008287e  _system_post_cinit             
1     00000400  __stack                        
1     00000500  __TI_STACK_END                 
1     0000a800  __TI_enable_exit_profile_output
1     0000a802  __TI_cleanup_ptr               
1     0000a804  __TI_dtors_ptr                 
1     0000a806  _lock                          
1     0000a808  _unlock                        
abs   00000100  __TI_STACK_SIZE                
abs   00000130  RamfuncsLoadSize               
abs   00000130  RamfuncsRunSize                
abs   ffffffff  __TI_pprof_out_hndl            
abs   ffffffff  __TI_prof_data_size            
abs   ffffffff  __TI_prof_data_start           
n/a   UNDEFED   __c_args__                     

[56 symbols]
